:020000000150AD
:02000300012DCD
:02000B00012EC4
:020013000143A7
:02001B0001439F
:02002300014397
:10002B00014332C0E0758AE8758C03758810E52BA7
:09003B00600314F52BD0E0323211
:10005000C2B375A8007581487580FF7590FF75A0C3
:10006000FF75B0F7C2B5C280C281C2827514F37544
:1000700015AF7516031208E97514D075150012082E
:10008000E47514D17515801208E4120A2B75A800C6
:10009000120BB47514F37515FF7516031208E912E7
:1000A0000D1511AC301DF8120A7480F330B2012224
:1000B0007514F41208EEE51420E03420E13220E259
:1000C0003020E32F20E42E20E52420E62120E7271E
:1000D0007514D07515001208E47514D175158012C9
:1000E00008E47514D87515021208E411F9222222C9
:1000F000222115411641AB4178C2017526E0752BCE
:1001000012752800750900750E007522017523000F
:10011000C21DD21E227514421208EE7514821208F6
:10012000EEE51430E50520E2358001227514021257
:10013000096F75250A7514F0120904E5156018B4E5
:100140000115E5267526E0B4320D8516407514F2CA
:1001500012096F120865227514F212096F227514C4
:100160000312096F7514F112096F7514F212096FF9
:1001700075140212096F7514F112096F75250A754D
:1001800014F01209047514F212096FE515B408741D
:10019000AA16AB17AC18AF19AD1AAE1CE51D600559
:1001A000752CFF80028E2CEB54F07058EA5420C35B
:1001B00013C0E0EB540FF526D0E04526C333F526F7
:1001C0009001C4736102614CA196618DA19661CECC
:1001D00061D1817481A781A881BA81BB81BCA196BC
:1001E000A196A196A19681BDA125A13BA196A1961C
:1001F000A196A196A196411041124114A196A196F3
:10020000A196A19612088412089002089C2241042B
:10021000A16DA16EA1787514431208EEE52654E095
:1002200064E0700122E526C2E0541F90022F73A102
:10023000A4C12C410EC17E410EC1D0C1F8E184E1C0
:1002400085E1ADE1C3E1DFE1EF410E410E410E4139
:100250000EE1F0E1F1E1F2410E410E410E410E419D
:100260000E417041724175410E410E410E410E2208
:10027000E1F30208030208137514471208EE75141F
:10028000871208EEE51420E5217514F07515007548
:100290001603854617854418854519752505753556
:1002A0000012094475440075450022751444120873
:1002B000EE7514841208EEE51420E5457514441219
:1002C00008EEE52B703BE53670377514F0751500B8
:1002D000751608853D1775180085371985381A85F4
:1002E000391B853A1C853B1D853C1E75250A7535D5
:1002F00000120938E537600122E53D6001227536BC
:100300000122EA5403603D14600F1460287526E052
:1003100012088412089002089C74204526F526EDE8
:10032000146009E53F440854FDF53F22E53F4402CF
:1003300054F7F53F2274404526F526ED540FC44589
:100340003FF53F2274004526F5262222EA54036039
:100350001214601C1460227526E0120884120890A2
:1003600002089CECB401F0C21E74004526F526225A
:10037000615774204526F52622ECB400DAED540FBF
:10038000C4453FF53F74404526F5262222EA540332
:10039000601214601C1460227526E0120884120892
:1003A0009002089CECB401F0D21E74004526F5269C
:1003B00022619874204526F52622ECB400DAED542B
:1003C0000FC4453FF53F74404526F52622228C2870
:1003D00022EF14700774004526F526221470077466
:1003E000204526F5262214700674404526F526146D
:1003F000701B74604526F526ED6009E53F440854FE
:10040000FDF53F22E53F440254F7F53F2214701CEE
:1004100074804526F526ED146009E53F440854FD37
:10042000F53F22E53F440254F7F53F22EFB4211B8C
:1004300074A04526F526ED6009E53F440854FDF516
:100440003F22E53F440254F7F53F22B4221B74C01B
:100450004526F526ED6009E53F440854FDF53F22A9
:10046000E53F440254F7F53F22B423047526E02209
:100470007526E022EC14700774004526F526221438
:10048000700774204526F526221470067440452610
:10049000F52614700774604526F52622147007743B
:1004A000804526F526222222EC600CD21D7514E828
:1004B0007515031208E422C21D222222227526E0AD
:1004C000ED1460167514F075150075160375170098
:1004D00075180075190002095022851927E527149F
:1004E000600614602D0208847514F07515007516E9
:1004F00008853D1775180085371985381A85391B09
:10050000853A1C853B1D853C1E75250A7535000204
:1005100009507514F07515007516017517007525CD
:1005200003020950227526E07514F0751500751642
:1005300001852B17752503020950227526E07514D5
:10054000F0751500751601751701752503ED600B23
:10055000E53F5404600E7517008009E53F540160C3
:1005600003751700E53F54F5F53F02095022851940
:100570002B7526E012086522ED6004780480E5788A
:1005800001E5186008E8453FF53F020865E8F455C5
:100590003FF53F0208657526E012088412089002B4
:1005A000089C2222E52620E0FAD2E0F52654E0C499
:1005B0009005C07514F07515007516027518007356
:1005C000A1C6A1D8A1EA7526E07402201E0254013A
:1005D000F5177525040209507526E0751700752575
:1005E00004E53F54F5F53F0209507526E0E53FC4A8
:1005F000540F60217514F0751500751602751800FA
:10060000751700B4011E7514841208EE5408600EAC
:1006100075170180097400A217334400F51775257A
:10062000040209507514871208EE80E0E52620E0E8
:100630004CD2E0F52654E0C490063C73C142C14957
:10064000C1501208657526E0221208657526E02261
:100650007526E0E53FC4540F600C14601414601755
:100660001208D8020865C2171208C01208B402089E
:10067000651208CC0208651208D802086522E52632
:1006800020E04CD2E0F52654E0C490068E73C1946D
:10069000C19BC1A21208657526E022120865752665
:1006A000E0227526E0E53FC4540F600C146014147A
:1006B00060171208A8020865D21712088412089061
:1006C00002086512089C0208651208A80208652243
:1006D000E52620E022D2E0F5267526E012086575B1
:1006E00014F41208EEE51430E3F57514D1E528444E
:1006F00080F5151208E42222E52620E007D2E0F575
:1007000026752A0054E0C490070B73E119E122E139
:100710002BE131E145E159E16D900D45752912025A
:100720000823900D5775293B0208237526E002081F
:1007300084E53F54087005900D608003900D797535
:100740002909020823E53F54087005900D728003C3
:10075000900D8B752907020823E53F54087005901A
:100760000D698003900D82752909020823E53F5425
:10077000087008900D9275293F8006900DD175295B
:100780003202082322E52620E022D2E0F526751465
:10079000F07515007516017517007525037526E0AF
:1007A000201D0302095075170102095022E5262079
:1007B000E010D2E0F5267526E0E5284480F5281201
:1007C000086522E52620E016D2E0F5267514F075BE
:1007D000150075160175170075250302095022E5ED
:1007E0002620E00AD2E0F5267526E01208652222CE
:1007F000222222E52620E00AD2E0F5267526E01224
:10080000086522E52620E00AD2E0F5267526E012EA
:10081000086522E52620E00AD2E0F5267526E002EA
:100820000884227514831208EEE51420E536751449
:10083000F0751500752500781779080525E52A93C8
:10084000052AF608E52AB52C067526E0020859B5F2
:1008500029057526E00159D9E27816A62505250552
:10086000251209502275140312096F7514F07515BD
:100870000075160075170075250312095A7514FACC
:1008800012096F2275144375150175250102095A65
:1008900075144275150175250102095A75144475C0
:1008A000150175250102095A75144775150175253D
:1008B0000102095A75144375150075250102095A7C
:1008C00075144275150075250102095A7514447591
:1008D000150075250102095A75144775150075250F
:1008E0000102095A752501215A752502215A7525DB
:1008F00001211BE514C0E0751400316F11EED0E04A
:10090000F5148017E514C0E0E525C0E07514023148
:100910006F11EED0E0F525D0E0F5147513367512A1
:1009200001318E751335852512317822D201751467
:1009300001316F7514F08022D201751404316F7586
:1009400014F08016D201751407316F7514F0800A07
:10095000D201751403316F7514F0316F751334853E
:10096000251231903001077514FA316FC2012275DA
:100970001336751201318E2285121131A720000A1B
:1009800078141209C1F608D511F8120A1F2278143A
:1009900085121131A720000BE61209F2082000038E
:1009A000D511F5120A1F22C20030B11230B00FC2A9
:1009B000B0120A2AC2B1120A2AE51331F222D20079
:1009C00022751008120A19120A2AA2B033C2B112F3
:1009D0000A2AD510EFC0E0E511B40104D2B08002BC
:1009E000C2B0120A19D0E0120A2AC2B1D2B0120A59
:1009F0002A227510083392B0120A19120A2AC2B1BB
:100A0000120A2AD510EFD2B0120A19120A2A30B0EF
:100A100002D200C2B1120A2A22D2B130B1FD22C2E2
:100A2000B05119512AD2B0512A22227536007524AC
:100A300000753F05758AE8758C0375890075881007
:100A400075A882753700753800753900753A0075DC
:100A50003B00753C00753D00754000753500752EF6
:100A600000752F0075300075310075320075330048
:100A70007534002251F2E5A0F46040AB24ACA079BB
:100A8000103024057524008002052451F2E5A0FAF7
:100A90007E01ECF45E600CEAF45E6007ECF45E4A02
:100AA000F4700CEEC3336003FE80E7D9D480068B6C
:100AB00024711B41BB8B2451F2713A20240305247D
:100AC000227590FF7580FFD2B4B115752400852E74
:100AD00037852F3885303985313A85323B85333C2F
:100AE00085343D515BE5477006D2B6D2B771BF91F0
:100AF0002B22D2B5D280D281D282E5242024137158
:100B000031D2B4202306F5907580FF227590FFF551
:100B100080227590FF7580FFC2B422752E01752F5B
:100B20000175300175310175320175330175350676
:100B300022E5245407900E039322E5A0752D08C3E7
:100B40003340027149D52DF822152DC0E0900E0BCF
:100B5000E52423232354F8452D936038F504900DA4
:100B6000347D08ED93B5040BED24089342347536BB
:100B7000006194DDEE7406B53504711B8016753680
:100B800000E9C0E0ECC0E0742E2535F9D0E0F7D0E4
:100B9000E0F9053530B318301E15E8C0E0EAC0E0D2
:100BA0007514F67515001208E4D0E0FAD0E0F8D01C
:100BB000E0052D22D2B7D2B67546007547002274E3
:100BC000F5918D500891E764FA700280012274F665
:100BD000918D91E764FA702B74E7918D91E764FA37
:100BE000702174E8918D91E764FA70177403918D08
:100BF00091E764FA700D74F4918D91E764FA7003D3
:100C00007547FF22741E800E7405800A740F8006DB
:100C10007421800274FF1470FD227FFF80027F1414
:100C200074A50000001470FADFF622D2B630B6FDCB
:100C300091E75031F54191E7502BF54291E750256E
:100C4000F543C2B6854244E543F404F545E5413039
:100C5000E00543460180035346FE30E1044346026B
:100C6000225346FD22E54714F547C2B6D2B722C04B
:100C7000E074FFC314600420B6FAD3D0E022C0E0D1
:100C800074FFC314600430B6FAD3D0E022D2B7C2E6
:100C9000B67900781400000000D8FAC2B7781400C2
:100CA000000000D8FAD2B6780820B604917E5032FF
:100CB000916F502E1392B7500109917E5024916F7D
:100CC0005020D8F0E913B392B7917E5015916F5030
:100CD00011D2B7917E500B916F5007917E5003D285
:100CE000B7D3D2B7D2B6227808916F5025917E50F3
:100CF0002120B71E916F501A917E5016A2B713D8BB
:100D0000F3916F50DD917E50D9916F50D5917E5007
:100D1000D1D3D2B722E540F413928013928213927A
:100D200081C2B52230313233343536373839414219
:100D30004344454600E1E5E0E4E2E6E3E702200162
:100D400010044080801201000100000008710402BC
:100D50000300010000000109023B00020100A005A0
:100D60000904000001030101000921000100012222
:100D70003F00070581030800120904010001030177
:100D80000200092100010001223200070582030848
:100D9000001205010906A101050719E029E7150060
:100DA0002501750195088102950175088101950558
:100DB0007501050819012905910295017503910135
:100DC0009506750815002565050719002965810038
:100DD000C005010902A1010901A1000509190129A4
:100DE00003150025019503750181029501750581A3
:100DF000010501093009311581257F7508950281AA
:100E000006C0C0FEFDFBF7EFDFBF7F4448463E3C17
:100E100042403A1823240D100E361C1221260A05D2
:100E20003338151320270919342C082F1F2D0706D6
:100E3000615E1A564F314E4B555B625751314D4AE8
:100E4000545A635250654C4953595800E30000000E
:100E500000000087948800E2E68B00E43900E0009F
:100E60000097008995E50096008AE128352A041D3F
:100E70005F5C2B301E2E161B605D144347453D29D9
:100E8000413F3B0C22250B110F37170000000000DB
:0B0E900000E700000000000000000070
:00000001FF
